:1000000009308A005B290000633479316100633470
:10001000793161006A3084008313000803191D28B8
:100020000230F800F701F70B1328F80B122897306D
:10003000F700F70B1928800B10280800A0132008E0
:1000400083168700831287130830F80027280000E2
:10005000F8173828F813ED0C03188717031C8713BB
:10006000781738287813F80B2B28362800008717C4
:100070003F308400840B3A280000F81B2A28781BA4
:1000800032280800831603178C170C140000000098
:1000900083120C087F39031986280313EA0003171B
:1000A0000D080313EB0003170F080313EC006A0895
:1000B000ED001E206B0803178D0003136C08031757
:1000C0008F0083168C170C140000000083120C0D97
:1000D0000E0D7F39031986280313EA0003170D0854
:1000E0000313EB0003170F080313EC006A08ED007D
:1000F0001E206B0803178D0003136C0803178F0075
:100100008D0A03198F0A03134228031703130800EB
:100110006908013A03199C28033A0319D028013AC7
:100120000319F428073A03191829013A03193C293D
:10013000033A0319602983298316881383128817C9
:1001400083160611831206158316851083128514F3
:1001500083168511831285156430EA000A20831600
:1001600008138312081383168813831288138316C7
:1001700006118312061183168611831286118316C7
:1001800005108312051083168510831285108316BF
:1001900005118312051183168511831285118B2990
:1001A0008316881383128817831606118312061587
:1001B0008316051083120514831685118312851585
:1001C0006430EA000A20831688138312881383168A
:1001D000061183120611831605108312051083166B
:1001E0008511831285118B29831688138312881732
:1001F0008316061183120615831685108312851443
:1002000083160511831205156430EA000A2083164F
:10021000881383128813831606118312061183161E
:1002200085108312851083160511831205118B2901
:1002300083160813831208178316061183120615F6
:1002400083168510831285148316851183128515F4
:100250006430EA000A2083160813831208138316F9
:1002600006118312061183168510831285108316DA
:100270008511831285118B298316881383128817A1
:1002800083168611831286158316051083120514B2
:1002900083168511831285156430EA000A208316BF
:1002A000881383128813831686118312861183168E
:1002B00005108312051083168511831285118B2971
:1002C0008316881383128817831686118312861566
:1002D0008316851083128514831605118312051564
:1002E0006430EA000A208316881383128813831669
:1002F000861183128611831685108312851083164A
:10030000051183120511043003178D0000308F0092
:10031000031342208B2908000830F80000008711E1
:10032000A0112008831687000000F10D8312071228
:10033000031CA0292016200883168700A4298312F5
:10034000201220088316870000008312A0152008C1
:10035000831687008312871DAB29F80B8E290000B6
:100360008711A01120088316870000008312201631
:10037000200883168700000000008312A0152008C3
:10038000831687008312871DC329F8010000071A0E
:1003900078148711A0112008831687008312071292
:1003A0002012200883168700831208006908013A8A
:1003B0000319F029033A0319F329013A0319F6291D
:1003C000073A0319F929013A0319FC29033A0319D9
:1003D000FF29013A0319022A0F3A0319052A082AAC
:1003E0000130E900102A0230E900102A0430E90047
:1003F000102A0830E900102A1030E900102A2030B5
:10040000E900102A4030E900102A8030E900102A63
:10041000073003178D0000308F0003134220102A8D
:10042000201620088316870000008312A0152008DC
:1004300083168700000083120712201220088316FB
:100440008700000083128711A011200883168700FF
:10045000E030F10083128C216908F1008C21201218
:1004600020088316870000008312A0152008831639
:1004700087008312871D3A2A00003E2A00002016BA
:100480002008831687000000831208000830F2005D
:100490007708F300201620088316870000008312D7
:1004A000A0152008831687008312871D552A071A76
:1004B0000314071E0310F80D0000A0112008831676
:1004C000870083128711F20B4A2A20162008831610
:1004D000870000008312071273080319742A201280
:1004E00020088316870083120000A01520088316B9
:1004F00087008312871D7A2A00008711A011200827
:10050000831687000000831207122012200883162A
:10051000870083120800EE01ED01201620088316E3
:10052000870000008312A0152008831687000000B2
:1005300083120712201220088316870000008312FE
:100540008711A011200883168700AA30F1008312BA
:100550008C216B08F1008C2120162008831687005F
:1005600000008312A0152008831687000000831264
:10057000871DB82A07122012200883168700000062
:1005800083128711A011200883168700AB30F10079
:1005900083128C21F70146227808F00020122008EF
:1005A0008316870000008312A01520088316870099
:1005B0008312871DD92A0000DD2A0000201620089A
:1005C00083168700000083122016200883168700F8
:1005D00000008312A01520088316870000008312F4
:1005E000071220122008831687000000831287114B
:1005F000A011200883168700AA30F10083128C21F5
:100600006C08F1008C21201620088316870000005A
:100610008312A01520088316870000008312871D0F
:100620000F2B071220122008831687000000831268
:100630008711A011200883168700AB30F1008312C8
:100640008C21F70146227808EF002012200883163B
:10065000870000008312A0152008831687008312EC
:10066000871D302B0000342B000020162008831635
:1006700087000000F20183126F08F100F200F1011F
:1006800070087107ED007208EE000318EE0A6D089D
:10069000F8006E08F90008000A30EB000B30EC009F
:1006A0008B227908EA007808E9006908F8006A08EE
:1006B000F90008000230EB000330EC008B227908CF
:1006C000EA007808E9006908F8006A08F9000800FB
:1006D0000830EB000930EC008B227908EA0078083A
:1006E000E9006908F8006A08F90008008E30F70090
:1006F0006A08F8006908F900FA01F808031D8A2B56
:100700007908F800F9010830F702F808031D8A2B70
:10071000F701922B0310F81B912BF90DF80DF7033D
:100720008A2BF81308006D0803196B2C8316A4009C
:100730007108031D9D2B83126B2CA402031CA72B95
:100740007F30A407031CA62B83126B2CB12B8130A6
:10075000A4020318AD2B83126B2C031DB12B831243
:100760006B2C2408F700F801F901FA01A3018312A8
:100770006E088316A200A21783126F088316A100C9
:100780007008A0001930A4007408A0020318D82B28
:100790000130A1020318D82BA2020318D82BA30200
:1007A0000318D82BA30AA20AA10A7408A0070A2CCE
:1007B0007308A1020318F32B0130A2020318F32BD4
:1007C000A3020318F32BA30AA20A7308A107740853
:1007D000A007031C0A2CA10A031D0A2CA20A031D50
:1007E0000A2CA30A0A2C72088038A2020318092CCA
:1007F0000130A3020318092CA30A72088038A2074B
:100800007308A107031CE72BA20A031DE72BA30A09
:10081000E72B7A14A40B0D2C182C0310A00DA10D9E
:10082000A20DA30D0310FA0DF90DF80DA50DC42BA3
:10083000251C202C0310F80CF90CFA0CA50C242C08
:10084000F70B242C83126B2CA51B4D2C0310A00D31
:10085000A10DA20DA30D7408A0020318392C0130BC
:10086000A1020318392CA2020318392CA302031C7D
:100870005E2C7308A1020318442C0130A202031855
:10088000442CA302031C5E2C72088038A2020318B9
:100890004D2C0130A302031C5E2CFA0A031D5E2CB2
:1008A000F90A031D5E2CF80A031D5E2CF70A031DCE
:1008B0005B2C83126B2CF80CF90CFA0C83126E086B
:1008C0008316A4007208A406A41F682CF817702CC5
:1008D000F813702C8312F701F801F901FA0183165D
:1008E000831208008E30F7007008F8006F08F900D6
:1008F000FA01F01F802CF809F909F90A0319F80A1E
:10090000F808031D8D2C7908F800F9010830F7026A
:10091000F808031D8D2CF701962C0310F81B942C5E
:10092000F90DF80DF7038D2CF01FF81308006F0870
:100930000319162D8316A0007308031DA12C831222
:10094000162DA0070318AF2C7F30A0020318AA2C85
:100950008312162D031DAE2C8312162DB52C81305B
:10096000A007031CB52C8312162D2008F700F801F0
:10097000F901FA017008A400A4177108A300720815
:10098000A2001830A000A101221CDE2C7608FA0774
:10099000031CD02CF90A031DD02CF80A0319A11747
:1009A0007508F907031CD72CF80A0319A117740856
:1009B000F100F1177108F8070318A117A10DF80C41
:1009C000F90CFA0CA40CA30CA20C0310A00BC32C62
:1009D0000130F707031CEE2C8312162DF81BF82CA0
:1009E000A40DFA0DF90DF80DF70BF82C8312162D46
:1009F000A41F0B2DFA0A031D0B2DF90A031D0B2D45
:100A0000F80A031D0B2DF80CF90CFA0CF70A031D5C
:100A10000B2D8312162D7008A1007408A106A11FCA
:100A2000132DF8171B2DF8131B2D8312F701F80156
:100A3000F901FA018316831208008E30F7006F085F
:100A4000F7027008F9007108F800F917F7080319A0
:100A5000342D0310F908031D302DF8080319342D27
:100A6000F90CF80CF70B292DF01F3B2DF809F909AB
:100A7000F80A0319F90A08000130E900D6214C23CD
:100A80007908A8007808A7005A237908A2007808F6
:100A9000A10068237908AE007808AD000230E900B3
:100AA000D6214C237908AA007808A9005A2379088E
:100AB000A4007808A30068237908B0007808AF0084
:100AC0000330E900D6214C237908AC007808AB004C
:100AD0005A237908A6007808A50068237908B2008F
:100AE0007808B1002E08EA002D08E900762377087F
:100AF000E9007808EA007908EB007A08EC00F000D9
:100B00007908EF007808EE007708ED00F401F301B2
:100B10007A30F2008830F10093232808EA00270891
:100B2000E9007708EB007808EC007908ED007A0816
:100B3000EE002808F0002708EF0072247A08F2007F
:100B40007908F1007808F0007708EF006E08F600E9
:100B50006D08F5006C08F4006B08F30097247A0820
:100B6000F2007908F1007808F0007708EF001D2501
:100B70007908B4007808B3003008EA002F08E900CB
:100B800076237708E9007808EA007908EB007A080C
:100B9000EC00F0007908EF007808EE007708ED002F
:100BA000F401F3017A30F2008830F10093232A082F
:100BB000EA002908E9007708EB007808EC007908DA
:100BC000ED007A08EE002A08F0002908EF007224F0
:100BD0007A08F2007908F1007808F0007708EF0051
:100BE0006E08F6006D08F5006C08F4006B08F30061
:100BF00097247A08F2007908F1007808F000770865
:100C0000EF001D257908B6007808B5003208EA0023
:100C10003108E90076237708E9007808EA007908C6
:100C2000EB007A08EC00F0007908EF007808EE009D
:100C30007708ED00F401F3017A30F2008830F1001A
:100C400093232C08EA002B08E9007708EB007808CA
:100C5000EC007908ED007A08EE002C08F0002B0873
:100C6000EF0072247A08F2007908F1007808F000A9
:100C70007708EF006E08F6006D08F5006C08F400C8
:100C80006B08F30097247A08F2007908F1007808DD
:100C9000F0007708EF001D257908B8007808B70044
:100CA00008006308840083136418831772088000A7
:100CB000840A8001E30A0319E40A0800F101040828
:100CC000F0007110831B7114EA1F6E2EF017701E56
:100CD000F00AE909EA09E90A0319EA0A6A0EF03892
:100CE000EC00EC07E23EED00323EEF006A080F39FF
:100CF000ED07ED07EF07E93EEE00EE07EE07690EA0
:100D00000F39EE07EF07EE0DEF0DEF09EF0D690854
:100D10000F39EF07EC0D0730EB000A30EF07EE0359
:100D2000031C8E2EEE07ED03031C922EED07EC0341
:100D3000031C962EEC07EB03031C9A2E6B308400E9
:100D4000831307307005701384037005031DAF2EE5
:100D5000701A840A701AAF2E2030F700CC2E840748
:100D60006F300402031970170008F700031DC02E2E
:100D7000701BC02E701ADA2EF019C02E2030CB2E28
:100D8000F01FC82E2D30F70084037013F013CC2E03
:100D9000F01570123030F707EA010408E9006A1014
:100DA000831B6A147708F2005126690884008313B4
:100DB0006A188317840A701FB02E08008008031970
:100DC000F32EEA010408E9006A10831B6A14000884
:100DD000ED001E206908840083136A188317840AB3
:080DE0000319850ADE2E08004C
:1010000080308318F2068316A201A30183126E08B2
:101010008316A1007208A10683126D080319022924
:101020008316A000F700710803190C29A002031908
:10103000A228031C5A287208A600A6177308A50048
:101040007408A400A3010310A60CA50CA40CA30C07
:10105000A00B2228A11F2F2822142429221020109F
:10106000221670308400831339292212A11B4228D2
:10107000201C4D28A60CA50CA40CA30CF70A0319E0
:101080001F294D28A61B50280310A30DA40DA50D44
:10109000A60DF70303191F2942282217C42822137B
:1010A00083126E088316A100A11F5828A6171829BD
:1010B000A61318297108A000F70083126D08831683
:1010C000A00283126E088316A600A61783126F086B
:1010D0008316A5007008A400A3010310A60CA50C9C
:1010E000A40CA30CA00B6C28A11F7928A2142429FE
:1010F000A2102010A2167430840083133929A21282
:10110000A11B8C28201C9728A60CA50CA40CA30CB2
:10111000F70A03191F299728A61B9A280310A30D65
:10112000A40DA50DA60DF70303191F298C28A217DE
:10113000C428A2137208A100A11FA028A61718296D
:10114000A61318297208A600A6177308A50074082C
:10115000A400A11FAF28A613221524292211A30140
:1011600020107030840083133929A11BDA288312E0
:101170006E088316A100201CC428A60CA50CA40C84
:10118000A30CF70A03191F29A31FD528A40A031DBE
:10119000D528A50A031DD528A60A031DD528A60C07
:1011A000A50CA40CF70A03191F29221B4F28A21B08
:1011B0009928FB288030A606A61FE2282429720859
:1011C000A100F12883126E088316A100A608031D52
:1011D000F128A508031DF128A408031DF128F70133
:1011E0001829A61BFB280310A30DA40DA50DA60D01
:1011F000F70BF1281F29A11FFF28A6171829A613EE
:10120000182983127108F70072088316A600730864
:10121000A5007408A400182983126D08F7006E0851
:101220008316A60083126F088316A5007008A40019
:101230002608F8002508F9002408FA005729F701C4
:10124000F801F901FA015729A301A409A509A60982
:10125000A309A30A031D3229A40A031D3229A50AE2
:101260000319A60A22182E28A21878282219AE28B7
:10127000DF280008A407031C4329A50A031D4329EE
:10128000A60A0319201484030008A507031C4B2990
:10129000A60A0319201484030008801F803AA607B9
:1012A00003182014221A3528A21A7F28B528831281
:1012B0008A150A12952C840183131F30830571301F
:1012C00083168F000F088312A0132008831687004F
:1012D00083128717831603170908C039890003137F
:1012E0001F129F12003003178800831287018801A4
:1012F0008901FF300313A000E301E4010130E9009C
:101300008A1188208A15831603170908C0398900B5
:1013100003131F129F120030031788008312031358
:101320001F139F1383169F1383121F149412A0126E
:101330002008831687008312201620088316870052
:101340008312A011200883168700013083129400B5
:101350000030831694000108C739083881008312D1
:1013600090010030F8009200003083169200831242
:1013700020152008831687008312970183169B018E
:101380009C0101309D0083120317870188018901A8
:101390000313E9008A1188208A158A113C258A15D1
:1013A000A208031D6C2A2108133C031C6C2AA40804
:1013B000031DDE2923080A3C0318E4290330E90051
:1013C0008A1188208A15F629A608031DEB2925080D
:1013D0000A3C0318F1290230E9008A1188208A1595
:1013E000F6290430E9008A1188208A158A113C25E3
:1013F0008A15E4013B30E3002030F2008A115126C7
:101400008A15033084002208EA002108E9008A11C5
:101410005E268A152030F2008A1151268A15033083
:1014200084002408EA002308E9008A115E268A1550
:101430002030F2008A1151268A15033084002608D4
:10144000EA002508E9008A115E268A152030F2009C
:101450008A1151268A15013084003408EA003308C5
:10146000E9008A115E268A152030F2008A11512681
:101470008A15013084003608EA003508E9008A112F
:101480005E268A152030F2008A1151268A15013015
:1014900084003808EA003708E9008A115E268A15B8
:1014A0002030F2008A1151268A1501308400EA01A9
:1014B000E9018A115E268A153B30840083138A1164
:1014C000DE268A151430E900FA30EA008A110A2073
:1014D0008A15E90B642AD029A408031D732A23085E
:1014E000603C0318012BA208031D7A2A2108623CE4
:1014F0000318802A0630E9008A1188208A15852A77
:101500000330E9008A1188208A158A113C258A1542
:10151000E4013B30E3002030F2008A1151268A15A5
:10152000033084002208EA002108E9008A115E26BF
:101530008A152030F2008A1151268A150330840062
:101540002408EA002308E9008A115E268A15203063
:10155000F2008A1151268A15033084002608EA0019
:101560002508E9008A115E268A152030F2008A11CA
:1015700051268A15013084003408EA003308E90056
:101580008A115E268A152030F2008A1151268A15AA
:10159000013084003608EA003508E9008A115E2629
:1015A0008A152030F2008A1151268A1501308400F4
:1015B0003808EA003708E9008A115E268A152030CB
:1015C000F2008A1151268A1501308400EA01E901EE
:1015D0008A115E268A153B30840083138A11DE2629
:1015E0008A150230A3020030031C0130A40214301B
:1015F000E900FA30EA008A110A208A15E90BF92A73
:101600006C2AA608031D082B2508603C0318962B9E
:10161000A208031D0F2B2108623C0318152B05306F
:10162000E9008A1188208A151A2B0230E9008A11F4
:1016300088208A158A113C258A15E4013B30E30095
:101640002030F2008A1151268A15033084002208C6
:10165000EA002108E9008A115E268A152030F2008E
:101660008A1151268A15033084002408EA002308D1
:10167000E9008A115E268A152030F2008A1151266F
:101680008A15033084002608EA002508E9008A113B
:101690005E268A152030F2008A1151268A15013003
:1016A00084003408EA003308E9008A115E268A15AE
:1016B0002030F2008A1151268A1501308400360844
:1016C000EA003508E9008A115E268A152030F2000A
:1016D0008A1151268A15013084003808EA0037083B
:1016E000E9008A115E268A152030F2008A115126FF
:1016F0008A1501308400EA01E9018A115E268A1503
:101700003B30840083138A11DE268A150230A5023D
:101710000030031C0130A6021430E900FA30EA0060
:101720008A110A208A15E90B8E2B012B8316861449
:101730008312861C5D2C8A113C258A15A208031D84
:10174000C82B2108613C031CC82BA408031DAC2B2B
:101750002308143C0318B22B0330E9008A118820B7
:101760008A15C42BA608031DB92B2508143C0318A1
:10177000BF2B0230E9008A1188208A15C42B013062
:10178000E9008A1188208A158A113C258A15E72BE1
:10179000A408031DCF2B2308143C0318D52B0630B7
:1017A000E9008A1188208A15E72BA608031DDC2B87
:1017B0002508143C0318E22B0530E9008A11882023
:1017C0008A15E72B0130E9008A1188208A158A11D1
:1017D0003C258A15E4013B30E3002030F2008A11F9
:1017E00051268A15033084002208EA002108E90006
:1017F0008A115E268A152030F2008A1151268A1538
:10180000033084002408EA002308E9008A115E26D8
:101810008A152030F2008A1151268A15033084007F
:101820002608EA002508E9008A115E268A1520307C
:10183000F2008A1151268A15013084003408EA002A
:101840003308E9008A115E268A152030F2008A11D9
:1018500051268A15013084003608EA003508E9006F
:101860008A115E268A152030F2008A1151268A15C7
:10187000013084003808EA003708E9008A115E2642
:101880008A152030F2008A1151268A150130840011
:10189000EA01E9018A115E268A153B308400831330
:1018A0008A11DE268A151430E900FA30EA008A111E
:1018B0000A208A15E90B552C962B0130E9008A1174
:1018C00088208A15B508031D6D2CB608031D6D2CE4
:1018D0002730BA000F30B900E92C3808F00037087B
:1018E000EF008A1172248A157708E9007808EA0067
:1018F0007908EB007A08EC003608F0003508EF00B4
:101900008A1172248A1583146C08F0006B08EF00AA
:101910006A08EE006908ED007A08F4007908F3001F
:101920007808F2007708F10000287708E9007808C5
:10193000EA007908EB007A08EC003608F000350878
:10194000EF008A1172248A156C08F0006B08EF0012
:101950006A08EE006908ED007A08F4007908F300DF
:101960007808F2007708F1008A1193238A15770826
:10197000E9007808EA007908EB007A08EC00F20048
:101980007908F1007808F0007708EF00F601F5011A
:101990004830F4008530F3008A1197248A157A08BC
:1019A000E8007908E7007808E6007708E5006808AD
:1019B000F2006708F1006608F0006508EF008A1180
:1019C0001D258A15FA017808F81BFA03B9007A0870
:1019D000BA00E4013B30E3002030F2008A115126C6
:1019E0008A15033084002208EA002108E9008A11E0
:1019F0005E268A152030F2008A1151268A1503309E
:101A000084002408EA002308E9008A115E268A156A
:101A10002030F2008A1151268A15033084002608EE
:101A2000EA002508E9008A115E268A152030F200B6
:101A30008A1151268A15013084003408EA003308DF
:101A4000E9008A115E268A152030F2008A1151269B
:101A50008A15013084003608EA003508E9008A1149
:101A60005E268A152030F2008A1151268A1501302F
:101A700084003808EA003708E9008A115E268A15D2
:101A80002030F2008A1151268A15013084003A086C
:101A9000EA003908E9008A115E268A153B30840085
:101AA00083138A11DE268A155030E900FA30EA00E5
:0E1AB0008A110A208A15E90B562DCD296300F4
:04400E00F52CFF3F4F
:00000001FF
